:1000000015C039C038C0DDC136C035C034C033C0BA
:1000100032C031C030C02FC02EC02DC02CC02BC06C
:100020002AC029C028C07000DB01510311241FBE63
:10003000CFE5D4E0DEBFCDBF10E0A0E6B0E0E4ED58
:10004000FCE002C005900D92A437B107D9F711E08A
:10005000A4E7B0E001C01D92AF30B107E1F710E0B6
:10006000CCE2D0E003C02297FE012FD6C632D107E2
:10007000D1F73CD02EC6C4CF0F931F93019769F5DB
:100080006F5F7F4F51F520E042E064E484E790E049
:1000900000D120E043E064E48CE790E0FAD00CE289
:1000A00011E02CED35E041E064E770E084E890E099
:1000B000E1D32CED35E040E06CE770E084E990E0BE
:1000C000D9D320E042E063E484EA90E098D020E0D5
:1000D00043E063E48CEA90E092D01F910F91089581
:1000E0006FEF7FEF81E090E0C7DF0895CF92DF925E
:1000F000EF92FF920F931F93CF93DF93F8D068EEA8
:1001000073E096D184E8C82E80E0D82EC4E9D0E010
:10011000EED0F4D07B018C018091AB00882371F18B
:10012000E091A500F091A600208130E08091A4002C
:1001300090E028233923232B09F161E07FEFC601EA
:1001400046D361E07FEFCE0142D3D1D028EE33E039
:10015000B801A701DFD0882381F36FEF70E0C601FB
:1001600036D361E07FEFCE0132D3C1D02CED35E044
:10017000B801A701CFD08823D9F5EFCF8091B30084
:10018000882371F1E091AD00F091AE00208130E064
:100190008091AC0090E028233923232B09F161E002
:1001A0007FEFC60114D361E07FEFCE0110D39FD063
:1001B00028EE33E0B801A701ADD0882381F361E0D8
:1001C0007FEFC60104D36FEF70E0CE0100D38FD074
:1001D0002CED35E0B801A7019DD0882349F4EFCF7D
:1001E0006FEF70E0C601F3D26FEF70E0CE01EFD297
:1001F0007ED0A801970164E170E0B2D089CF1F934F
:10020000CF93DF93EC01122F14D48F81882379F0E0
:10021000CE018DD4EB81FC819881112321F0808166
:10022000892B808304C08081909598239083DF91EF
:10023000CF911F9108951F93CF93DF93EC01122F5D
:10024000F8D38F81882379F0CE0171D4EB81FC81C2
:100250009881112321F08081892B808304C08081C3
:10026000909598239083DF91CF911F910895FC0181
:100270008781882369F0A381B4819081662321F06E
:100280008C91892B8C9308958C91909598239C93B5
:1002900008951F93CF93DF93EC01122FCAD38F8160
:1002A000882329F0CE0154D4612FCE01E0DFDF9105
:1002B000CF911F9108951F93CF93DF93EC01122FDD
:1002C000B8D38F81882329F0CE0142D4612FCE018B
:1002D000CEDFDF91CF911F91089514BC8AE085BDD8
:1002E0008DE783BD89B7806889BF7894089584EBD2
:1002F00090E00895F2DF0895F0DF08952FB7F894A5
:100300006091B5007091B6008091B7009091B800EF
:100310002FBF0895EF92FF920F931F937A018B01E5
:100320006FB7F8948091B5009091B600A091B70096
:10033000B091B8006FBF60E070E08E199F09A00B0C
:10034000B10B40E050E0281739074A075B0710F46B
:1003500061E070E0CB011F910F91FF90EF90089545
:10036000EF92FF920F931F9379018A01AB0160E036
:1003700070E02FB7F8948091B5009091B600A091ED
:10038000B700B091B8002FBF8E199F09A00BB10B19
:10039000481759076A077B0760F71F910F91FF9075
:1003A000EF900895019731F46F5F7F4F19F484EB5C
:1003B00090E0A2DF08956FEF7FEF81E090E0F2DF41
:1003C00008951F920F920FB60F9211242F933F930F
:1003D0004F935F936F937F938F939F93AF93BF934D
:1003E000EF93FF938091B5009091B600A091B70074
:1003F000B091B8000196A11DB11D8093B5009093F6
:10040000B600A093B700B093B8001FD050D1FF91B1
:10041000EF91BF91AF919F918F917F916F915F917C
:100420004F913F912F910F900FBE0F901F901895F5
:10043000EFB7F8942091B5003091B6004091B70025
:100440005091B800EFBF8CDF089589EB90E00895DC
:10045000DC012FB7F89480E090E0FC01EE0FFF1F65
:10046000EE0FFF1FE80FF91FEA0FFB1F1382128226
:1004700011821082848301968031910571F7A05B0F
:10048000BF4F1D921D92FD011082118212821382B4
:100490002FBF0895DC012FB7F89480E090E0FC01B5
:1004A000EE0FFF1FEE0FFF1FE80FF91FEA0FFB1FF4
:1004B0001382128211821082848301968031910509
:1004C00071F7A05BBF4F1D921D92FD01108211823A
:1004D000128213822FBF0895EF92FF920F931F9302
:1004E000CF93DF93EC018B01BA01FFB6F894C05BA8
:1004F000DF4F5881C055D04020E0852F90E0FC01AF
:10050000EE0FFF1FEE0FFF1FE80FF91FEC0FFD1F8F
:1005100082819381892B39F02F5F203109F4B0C09B
:1005200051505F70EACF503108F0AAC0DE01AF5AD7
:10053000BF4F8C9190E0FC01EE0FFF1FEE0FFF1FED
:10054000E80FF91FEC0FFD1F82819381892B09F4BD
:100550008FC08C9190E0FC01EE0FFF1FEE0FFF1F8C
:10056000E80FF91FEC0FFD1F808191816817790753
:1005700008F47EC0EC9022C08D919C911197681771
:100580007907E0F0FD01848190E08217930711F470
:10059000E42E14C0FD018481E42E482F242F30E086
:1005A000D901AA0FBB1FAA0FBB1FA20FB31FAC0F0D
:1005B000BD1FFD0182819381892BF1F6852F90E08B
:1005C000DC01AA0FBB1FAA0FBB1FA80FB91FAC0FDE
:1005D000BD1FFD011383028311967C936E93548398
:1005E000FFEFEF1621F12E2D30E0F901EE0FFF1F86
:1005F000EE0FFF1FE20FF31FEC0FFD1F848190E051
:100600008217930721F08481FD01848305C0CF5AAE
:10061000DF4F5883C155D040F901EE0FFF1FEE0F99
:10062000FF1FE20FF31FEC0FFD1F548329C09E0133
:10063000205B3F4FF901808190E0FC01EE0FFF1F2E
:10064000EE0FFF1FE80FF91FEC0FFD1F8281938152
:10065000892B29F0F9018081FD01848305C0CF5ADF
:10066000DF4F5883C155D040C05BDF4F588308C06F
:10067000C05BDF4F4881C055D040EE24EA948ECF56
:10068000FFBEDF91CF911F910F91FF90EF900895E2
:10069000019731F46F5F7F4F19F489EB90E0FADE38
:1006A00008956FEF7FEF81E090E0F2DF08958F9281
:1006B0009F92AF92BF92CF92DF92EF92FF920F93F1
:1006C0001F93CF93DF935C0112DE18DE9B01AC0118
:1006D000F501EE5AFF4F80819181A281B3817901AA
:1006E0008A01E81AF90A0A0B1B0B09F44BC0808136
:1006F0009181A281B381281739074A075B0728F443
:100700000894E108F108010911092083318342832B
:100710005383F501E05BFF4FC0804F0124C0DC80B4
:1007200088819981A0E0B0E0E816F9060A071B0766
:1007300088F0EA81FB811B821A8219821882CC829E
:10074000D401DC92A081B1812D913C91CF01F901BE
:10075000099506C0888199818E199F09998388839C
:10076000CD1481F0CD2C8C2D90E0EC01CC0FDD1F51
:10077000CC0FDD1FC80FD91FCA0DDB1D8A819B81DD
:10078000892B69F6DF91CF911F910F91FF90EF9028
:10079000DF90CF90BF90AF909F908F900895FC0115
:1007A0008781882369F0A381B4819081662321F039
:1007B0008C91892B8C9308958C91909598239C9380
:1007C000089561E054DD089560E051DD0895CF9211
:1007D000DF92EF92FF920F931F93CF93DF93EC0181
:1007E000E0D16C018C818823D1F1ED80FE800F81F6
:1007F00018857DDD24E130E0B801A7018BDD882379
:1008000071F18B85882321F0D094C194D108D394C1
:100810002C853D858E859F858C01020F131F281B1B
:10082000390B4FEF50E061E07FEFC601B5D08C018E
:10083000FFB6F89489859A85C4DFC80164E170E049
:10084000DED1CB0161E070E07ED089859A85BCDF86
:10085000FFBE4DDD53DD6D837E838F8398878A8154
:100860009B81DF91CF911F910F91FF90EF90DF90CF
:10087000CF900895AF92BF92DF92EF92FF920F93C5
:100880001F93CF93DF93EC015B01D42E790170D1DC
:1008900084E690E099838883DB86FD86EC861F875B
:1008A0000E87F5018781882369F0BA86A986C5017C
:1008B0008BDF1DDD23DD6D837E838F839887CE01E3
:1008C0006CD102C01A861986DF91CF911F910F91CA
:1008D000FF90EF90DF90BF90AF900895AF92BF92DE
:1008E000DF92EF92FF920F931F93CF93DF93EC0170
:1008F0005B01D42E79013CD184E690E09983888312
:10090000DB86FD86EC861F870E87F50187818823AD
:1009100069F0BA86A986C50157DFE9DCEFDC6D8393
:100920007E838F839887CE0138D102C01A861986BC
:10093000DF91CF911F910F91FF90EF90DF90BF90CB
:10094000AF9008950895CF93DF93CDB7DEB7229788
:100950000FB6F894DEBF0FBECDBF9A83898389811D
:100960009A819C01629FC001639F900D729F900DC0
:10097000112403C089819A8101979A83898389818F
:100980009A81892BB9F722960FB6F894DEBF0FBE75
:10099000CDBFDF91CF9108954F925F926F927F927A
:1009A0008F929F92AF92BF92CF92DF92EF92FF927F
:1009B0000F931F932B015A0139017801E21AF30AB0
:1009C0000027F7FC0095102F9C01261B370B4427AE
:1009D00037FD4095542FC801B701F2D0A418B508CF
:1009E000CC24B7FCC094DC2CA60195011BD1882433
:1009F00077FC8094982C620E731E841E951EC30192
:100A00001F910F91FF90EF90DF90CF90BF90AF902C
:100A10009F908F907F906F905F904F900895681790
:100A200079070CF4BC01461757070CF4BA01CB0147
:100A30000895FC0181E090E002C0880F991F4A955B
:100A4000E2F7808381E08783643419F165342CF404
:100A5000623449F0633451F511C0633679F064367D
:100A6000C1F0623619F587E390E09683858386E3CB
:100A700090E09283818388E390E015C084E390E066
:100A80009683858383E390E09283818385E390E07E
:100A90000AC081E390E09683858380E390E09283AF
:100AA000818382E390E0948383830895178208957D
:100AB000FC0181E090E002C0880F991F4A95E2F79F
:100AC000808381E08783643419F165342CF46234C7
:100AD00049F0633451F511C0633679F06436C1F0E2
:100AE000623619F587E390E09683858386E390E08C
:100AF0009283818388E390E015C084E390E096833D
:100B0000858383E390E09283818385E390E00AC04C
:100B100081E390E09683858380E390E092838183F4
:100B200082E390E094838383089517820895CF939E
:100B3000DF93DC01EC018F81882339F0ED81FE81A8
:100B400090818C91809589238083DF91CF91089546
:100B5000CF93DF93DC01EC018F81882331F0ED81AD
:100B6000FE8180819C91892B8083DF91CF910895B4
:100B7000FC018EE690E091838083138212821482BE
:100B80000895FC018EE690E09183808313821282A7
:100B900014820895FC011482089521E0FC0124834D
:100BA00008950F931F938C01CB014FEF50E061E04C
:100BB0007FEF35DFF801938382831F910F910895B2
:100BC000629FD001739FF001829FE00DF11D649F31
:100BD000E00DF11D929FF00D839FF00D749FF00DBD
:100BE000659FF00D9927729FB00DE11DF91F639F5E
:100BF000B00DE11DF91FBD01CF011124089597FB30
:100C0000092E07260AD077FD04D027D006D0002071
:100C10001AF4709561957F4F0895F6F79095819538
:100C20009F4F089597FB092E05260ED057FD04D03F
:100C300028D00AD0001C38F4509540953095219565
:100C40003F4F4F4F5F4F0895F6F790958095709501
:100C500061957F4F8F4F9F4F0895AA1BBB1B51E19A
:100C600007C0AA1FBB1FA617B70710F0A61BB70B1C
:100C7000881F991F5A95A9F780959095BC01CD01C1
:100C80000895A1E21A2EAA1BBB1BFD010DC0AA1FCD
:100C9000BB1FEE1FFF1FA217B307E407F50720F0E5
:100CA000A21BB30BE40BF50B661F771F881F991F60
:100CB0001A9469F760957095809590959B01AC01A9
:100CC000BD01CF010895EE0FFF1F0590F491E02DB7
:040CD0000994FFCFB5
:100CD40000000000E703CD05CA0500000000A204DF
:040CE400CD05CA056B
:00000001FF
